:100000000C948F050C94AC050C94AC050C94AC05C9
:100010000C94AC050C94AC050C94AC050C94AC059C
:100020000C94AC050C94AC050C943B2A0C940D2B51
:100030000C9442250C94AC050C94AC050C94AC05C6
:100040000C94AC050C94AC050C94AC050C94AC056C
:100050000C94AC050C94CA250C94AC050C94AC051E
:100060000C94AC050C94AC050C94AC050C94AC054C
:100070000C94AC050C94AC050C94AC050C94AC053C
:100080000C94AC050C94AC050C94AC050C94AC052C
:100090000C94AC050C94AC050C94AC050C94AC051C
:1000A0000C94AC050C94AC050C94AC052E092E09EF
:1000B0005A095A09C209E009F80AF80AEB09840A40
:1000C000950A950A7A2BA12B992CA12B992CED2B13
:1000D000102C992C672C762C2B0014001A00080089
:1000E0001500170000001C0018000C00120013007F
:1000F0002D00296104001600070009000A00000015
:100100000B000D000E000F0033003400E1001D0055
:100110001B000600190005000551110010003600F3
:100120003700380028623500E000E200E300AA5DF5
:100130002C00E5002A00AB5D5000510052004F003A
:100140002B0014001A00090013000A0000000D0023
:100150000F0018001C0033002D0029610400150059
:1001600016001700070000000B00110008000C002B
:1001700012003400E1001D001B00060019000500FC
:1001800005510E0010003600370038002862350097
:10019000E000E200E300AA5D2C00E5002A00AB5D70
:1001A0005000510052004F002B0034003600370041
:1001B00013001C00000009000A00060015000F00D3
:1001C0002D00296104001200080018000C00000036
:1001D00007000B001700110016003800E100330083
:1001E00014000D000E001B000551050010001A0040
:1001F00019001D0028623500E000E200E300AA5D5E
:100200002C00E5002A00AB5D5000510052004F0069
:1002100035021E021F0220022102220200002302D8
:1002200024022502260227024C004C003A003B0023
:100230003C003D003E0000003F002D022E022F0238
:1002400030023102010040004100420043004400FE
:10025000010045004D000100010001000100010006
:100260000100010001000100010001000100010086
:10027000AB00AA00A900AE0035001E001F00200040
:100280002100220000002300240025002600270072
:100290004C004C003A003B003C003D003E0000009A
:1002A0003F002D002E002F003000310001004000E3
:1002B0004100420043004400010045003200640058
:1002C0000100010001000100010001000100010026
:1002D0000100010001000100AB00AA00A900AE006E
:1002E00035021E021F022002210222020000230208
:1002F00024025200260227024C004C003A003B0028
:100300003C003D003E0000003F00500051004F0007
:10031000300231020100400041004200430044002D
:10032000010045004D000100010001000100010035
:100330000100010001000100010001004E004B001E
:10034000AB00AA00A900AE00000000000000000001
:10035000000000000000000000000000000000009D
:10036000000000000000000000000000000000008D
:10037000000000000000000000000000000000007D
:10038000000000000000000000000000000000006D
:1007500000000000000000000100005CC35CC45CFD
:10076000C75CC65C0000C95CC85CCB5CCA5C0100AD
:100770004C000100010001001D5C1E5C135C0000C8
:100780000A5CA75DA85DA95D0100010001002B5C6A
:100790002A5C265C275C2C5C01002D5C01000100BA
:1007A0000100010001000100010001000100010041
:1007B0000100010001000100010001000100010031
:1007C00000047F3F1F643214643214783C1E1E14F0
:1007D0000A052223252628292A2C2D2F30323335AD
:1007E00036383A3B3D3E4042434547494A4C4E50DD
:1007F00051535557595A5C5E6062646668696B6D07
:100800006F71737577797B7D7F81838587898A8C0A
:100810008E90929496989A9C9E9FA1A3A5A7A8AA11
:10082000ACAEAFB1B3B4B6B8B9BBBCBEBFC1C2C346
:10083000C5C6C7C9CACBCCCDCED0D1D2D2D3D4D5E0
:10084000D6D7D7D8D9D9DADADBDBDBDCDCDCDCDC09
:10085000DDDDDDDDDCDCDCDCDCDBDBDBDADAD9D9E1
:10086000D8D7D7D6D5D4D3D2D2D1D0CECDCCCBCA6F
:10087000C9C7C6C5C3C2C1BFBEBCBBB9B8B6B4B395
:10088000B1AFAEACAAA8A7A5A3A19F9E9C9A98962B
:100890009492908E8C8A89878583817F7D7B7977FE
:1008A0007573716F6D6B6968666462605E5C5A59DE
:1008B00057555351504E4C4A4947454342403E3D9F
:1008C0003B3A3836353332302F2D2C2A292826252D
:1008D0002322FFAA7F55400001010101010101010E
:1008E00001020202020202020202030303030303E3
:1008F00003030404040404040405050505050606B1
:10090000060606070707070708080808090909096E
:100910000A0A0A0B0B0B0C0C0C0D0D0D0E0E0E0F14
:100920000F0F1010111111121213131414151516A4
:10093000161717181819191A1A1B1B1C1D1D1E1E15
:100940001F20202122222324242526262728292966
:100950002A2B2C2D2D2E2F30313232333435363791
:1009600038393A3B3C3D3E3F40414243444546478F
:1009700048494A4C4D4E4F50515354555658595A68
:100980005B5D5E5F616264656668696B6C6D6F700C
:1009900072737577787A7B7D7E8082838587888A7B
:1009A0008C8E8F91939596989A9C9EA0A2A3A5A7B2
:1009B000A9ABADAFB1B3B5B7BABCBEC0C2C4C6C9AE
:1009C000CBCDCFD1D4D6D8DBDDDFE2E4E7E9EBEE67
:1009D000F0F3F5F8FAFDFF2603410074007200659C
:1009E000007500730020003500300020004B0065CA
:1009F00000790062006F0061007200640000001066
:100A00000348006500780077006900720065000007
:100A1000000403090409023B00020100A0FA0904D2
:100A20000000010301010009211101000122400021
:100A3000070581030800010904010001030000000B
:100A4000092111010001227B00070582032000011A
:100A5000120100020000000880BB0D040100010229
:100A6000000105010902A10185020901A100050992
:100A70001901290815002501950875018102050154
:100A8000093009311581257F9502750881060938DD
:100A90001581257F950175088106050C0A38021518
:100AA00081257F950175088106C0C005010980A1D7
:100AB00001850319012AB700150126B700950175B4
:100AC000108100C0050C0901A101850419012AA0AB
:100AD00002150126A002950175108100C0050109CB
:100AE00006A101050719E029E715002501950875FC
:100AF0000181029501750881010507190029FF157B
:100B00000026FF00950675088100050819012905D2
:100B1000950575019102950175039101C00011249D
:100B20001FBECFEFDAE0DEBFCDBF11E0A0E0B1E045
:100B3000E8E9FBE502C005900D92A43CB107D9F7A6
:100B400022E0A4ECB1E001C01D92A53DB207E1F79F
:100B50000E94E8160C94CA2D0C940000769A0C940E
:100B60000F06CF93DF93EC010E94D111BE0180E00C
:100B700090E0DF91CF910C94E00BCF93FB01893A89
:100B80002DE5920701F140F4873A2DE5920769F0CF
:100B9000883A9D4581F03FC08B3A2DE59207E1F000
:100BA000C0F08D3A9D4561F136C0C281CC23A1F1E0
:100BB00081E090E005C0C281CC2371F182E090E039
:100BC0000E94B10523C0C281CC2331F184E090E0C2
:100BD000F7CFC28183E002C0C28184E0CC2341F020
:100BE0000E94400C40E164E083E00E94B4060EC025
:100BF0000E94610C40E164E083E00E94B4060CC0F6
:100C0000C28185EECC2321F00E94AE07C0E004C073
:100C10000E945D0801C0C1E08C2FCF910895089516
:100C200081E008950C94BD0508950C9414061F935B
:100C3000CF93DF9300D000D01F92CDB7DEB74983AA
:100C40005A836B833091C70189819A81311114C015
:100C5000662359F0222349F00E94350D182F682F82
:100C600089819A810E94DE0C03C00E94090D182F11
:100C700069817A81812F04C00E94350D69817A8152
:100C80000F900F900F900F900F90DF91CF911F91C9
:100C90000C946E14FC01262F408151816281738176
:100CA00084810C94170681E00895CF93DF93EC01C3
:100CB00060E00E944A06BE01DF91CF910C941506B8
:100CC0008F929F92AF92BF92CF92DF92EF92FF925C
:100CD0000F931F936B017C0181E090E0A0E0B0E0F6
:100CE0004C015D0104C0880C991CAA1CBB1C4A95D0
:100CF000D2F7AC01BD0104C0440F551F661F771F1A
:100D00002A95D2F7482959296A297B2904C0880FD6
:100D1000991FAA1FBB1F0A95D2F78A019B010C21BC
:100D20001D212E213F21401751076207730739F417
:100D3000BC01CD016C297D298E299F290AC080958F
:100D40009095A095B095BC01CD016C217D218E219F
:100D50009F211F910F91FF90EF90DF90CF90BF9058
:100D6000AF909F908F9008950F93382F262F60910A
:100D7000EB017091EC018091ED019091EE01042F57
:100D8000432F0E9460060F910C941A0C0C94AE0530
:100D90000C94991508950E94880B0E94CA062FEFA3
:100DA00084E39CE0215080409040E1F700C00000C7
:100DB0000C94F0250F931F93CF93DF938C0161E088
:100DC0000E944A06EC01B8010E941206882309F429
:100DD00044C0B801CE010E940D248823F1F1B8016E
:100DE000CE010E94AA208823C1F1B801CE010E9441
:100DF0006923882391F1B801CE010E94B01F882396
:100E000061F1F8018281882309F1CB358DE5D8079E
:100E1000C1F050F4C115FCE5DF0781F0CF3DDC45A2
:100E2000A9F40E946B1219C0CC35EDE5DE0761F024
:100E3000CD35DD4559F40E94AF1108C00E94CB06A4
:100E40000CC00E94B81102C00E94BB11C801DF9102
:100E5000CF911F910F910C94100680E0DF91CF91FC
:100E60001F910F9108950E9424250C944C070E9415
:100E70004F070C942A2508950C943B0781E00895B0
:100E80000C943E070895CF93C82F0E943C078C2FE7
:100E90000E944007CF91089580E00C9443070E9480
:100EA00069240C9443070E9469249091C601891714
:100EB00021F08093C6010C9443070895CF93DF93EC
:100EC000CDB7DEB72B970FB6F894DEBF0FBECDBF00
:100ED0004F83588769877A878B8761110E94FB103F
:100EE0009E012F5F3F4F86E0F90111928A95E9F745
:100EF00085E0FE013796D90101900D928A95E1F7C0
:100F000089819A814C815D81452B31F09F3F31F47D
:100F100091E08F3F19F403C091E001C090E090FF91
:100F200009C049815A816B817C818D819E810E949B
:100F30001C1005C0C9010E9453068111F2CF2B96E7
:100F40000FB6F894DEBF0FBECDBFDF91CF910895ED
:100F5000FC01808191810E94770D0895CF938823B1
:100F600009F4A9C0C82F8238C1F40E94692481FD08
:100F7000A2C069E380910201909103010E94FC24C8
:100F80000E941D112FEF81EE94E02150804090408F
:100F9000E1F700C0000069E319C0833801F50E9441
:100FA000692480FD88C063E580910201909103016E
:100FB0000E94FC240E941D112FEF81EE94E021502D
:100FC00080409040E1F700C0000063E5809102019D
:100FD000909103010E94FE24CF910C941D1184383E
:100FE000C1F40E94692482FD66C067E48091020119
:100FF000909103010E94FC240E941D112FEF81EEAD
:1010000094E0215080409040E1F700C0000067E488
:10101000DDCF8CEF8C0F813AF8F48C2F0E942023C7
:10102000811149C06C2F80910201909103010E94AF
:10103000C624882349F06C2F80910201909103010E
:101040000E94FE240E941D116C2F8091020190913C
:1010500003010E94FC24C0CF80E28C0F883048F44A
:10106000C77081E001C0880FCA95EAF70E94DE10C0
:10107000B3CFEBE5EC0FE33040F4F0E0E65AFE4F7F
:10108000808190E0CF910C948E24E8E5EC0FE7315D
:1010900050F4F0E0EE0FFF1FE45DFE4F8081918180
:1010A000CF910C94A424CD3E30F08C2F0E946D176C
:1010B000CF910C943F18CF910895882309F464C010
:1010C000823879F40E94692481FF5EC069E38091CF
:1010D0000201909103010E94FC240E941D1169E30A
:1010E00010C08338B1F40E94692480FF4DC063E5CD
:1010F00080910201909103010E94FC240E941D1125
:1011000063E580910201909103010E94FE240C94FA
:101110001D11843879F40E94692482FF35C067E488
:1011200080910201909103010E94FC240E941D11F4
:1011300067E4E7CF9CEF980F913A10F4682FE1CF66
:1011400090E2980F983050F4877091E001C0990FA9
:101150008A95EAF7892F0E94E410D9CF9BE5980F72
:10116000933020F480E090E00C948E2498E5980F62
:10117000973120F480E090E00C94A4248D3E20F080
:101180000E94C8170C943F1808951F93CF93DF93C4
:10119000182FEB010E94AE07209741F08FE99FE0E6
:1011A0000197F1F700C000002197F6CF812FDF9162
:1011B000CF911F910C945D08893319F060E070E0C5
:1011C00002C060E570E00C94C508882321F00E94FD
:1011D000DE100C941D110895882321F00E94E41064
:1011E0000C941D110895CF92DF92EF92FF920F930E
:1011F0001F93CF93DF937C01D62FC72FFC01128161
:10120000058102950F700E94D4108823B9F0112334
:10121000A9F08C2F807F803421F080E28D0F883000
:1012200068F080918A0282FD09C082E00E947D11EF
:101230000E94D41091E0D82ED92601C0D12CCC2EFA
:10124000C2948FE0C8228C2D90E08C30910508F07C
:10125000CFC1FC01EA5AFF4F0C94252D8C2F807FC3
:10126000CF70882311F0C295C07F112399F0CC2351
:1012700009F4AAC180E28D0F883010F0D11104C0AA
:101280008C2F0E94DE1003C08C2F0E94EE100E9453
:101290001D119AC18D2F0E945D08CC2309F4A8C1AD
:1012A00080E28D0F883038F1DD2329F18C2F0E94E8
:1012B000F41024C08C2F807FCF70803211F0C29543
:1012C000C07FDD2319F0D130A1F13DC080918A02A9
:1012D00082FF17C0112349F0CC2329F08C2F0E94E4
:1012E000DE100E941D1180E070C180E00E945D0848
:1012F000CC2309F47DC18C2F0E94E4100E941D11A3
:1013000077C1112371F0002341F0013031F40E94C4
:10131000FE108C2B0E9406116BC10E94FE108C2BBC
:101320001DC0002319F0013009F462C10E9413119D
:1013300025C0112321F0063008F05AC10EC0053037
:1013400008F056C11BC0112361F0002331F0F701F2
:10135000858180FF39C18F7085838C2F0E94E508BD
:1013600047C1002359F0D93309F03FC1FFEF07EE21
:1013700013E0F15000401040E1F735C18C2F0E947E
:10138000EC0836C18C2F86958695837019F08130D4
:1013900061F02EC1112321F08D2F9C2F937002C07C
:1013A00080E090E00E948E242BC1112321F08D2F2C
:1013B0009C2F937002C080E090E00E94A42420C182
:1013C0008D2F112319F00E946D1702C00E94C817BB
:1013D0000E943F1815C18C2F837009F047C011116E
:1013E0000BC12D2F229526952770220F220F6D2FCE
:1013F0006F70862F90E0A0E0B0E0022E04C0880F4E
:10140000991FAA1FBB1F0A94D2F7D4FF10C04FE048
:1014100050E060E070E004C0440F551F661F771F66
:101420002A95D2F7409550956095709503C040E09D
:1014300050E0BA01C695C695C3708A019B01082B7E
:10144000192B2A2B3B2BC901B801C23049F058F4A3
:10145000C13019F00E94F40BCFC00E94E20BCCC047
:101460000E94060CC9C00E94E00BC6C0112319F0EF
:101470008C2F817001C08695882309F4BDC02D2F63
:10148000229526952770220F220F6D2F6F70862FC1
:1014900090E0A0E0B0E0022E04C0880F991FAA1FC0
:1014A000BB1F0A94D2F7D4FF10C04FE050E060E0B9
:1014B00070E004C0440F551F661F771F2A95D2F7AE
:1014C000409550956095709503C040E050E0BA019A
:1014D000C695C695C3708A019B01082B192B2A2B30
:1014E0003B2BC901B801C23049F058F4C13019F0A2
:1014F0000E94B90C81C00E94A70C7EC00E94CB0C38
:101500007BC00E941A0C78C0CF70112339F08C2F49
:101510000E94400C8D2F0E94E5086EC08D2F0E9406
:10152000EC088C2F0E94610C67C0D23F21F128F497
:10153000D03F41F0D13FC1F043C0D33F19F1D43F78
:1015400079F03EC0112341F0053008F051C08C2FD6
:101550008F710E94860C4CC0063008F049C0F7CF4E
:1015600080918A0282FF18C0112339F08C2F8F716D
:101570000E94400C3DC01123C9F38C2F8F710E9433
:10158000610C36C0112329F08C2F8F710E942B0C17
:101590002FC00E94260C2CC0112349F0CF718C2F34
:1015A0000E94400C63E08C2F0E94621121C081E0F8
:1015B0000E947D110230E0F082E00E947D1118C08F
:1015C000112331F0002391F28D2F0E94AE0710C03D
:1015D000002399F2D93349F41FEF27EE33E011507D
:1015E00020403040E1F700C000008D2F0E945D08D0
:1015F00088EF8C0D843020F40E9469240E944307F8
:10160000DD20C9F00E94D01080FD15C0F7011282C4
:101610000E94CA100E94400CC7010E943C0B0E940D
:10162000CA10DF91CF911F910F91FF90EF90DF9043
:10163000CF900C94610CDF91CF911F910F91FF908F
:10164000EF90DF90CF9008950F931F93CF93DF9388
:10165000EC01688179818A810E94820D8C010E944F
:10166000DD0C0E94CE0BB801CE010E94F308DF9181
:10167000CF911F910F910895CF93DF93EC01988143
:1016800089812B813C81232B31F08F3F31F481E024
:101690009F3F19F403C081E001C080E080FD1DC0C0
:1016A000CE010E94DA06811110C00E94D410882356
:1016B000A1F08A81882389F080918A0282FD0DC081
:1016C00082E0DF91CF910C947D11CE010E94240B1A
:1016D000CE01DF91CF910C945506DF91CF91089503
:1016E00080E090E00E948E2480E090E00E94A4249C
:1016F0000E94FB100E941D110E9470190C943F184B
:1017000080910201909103010E9400250C94700BBE
:101710000E94EB100C94800B92959F70963079F09C
:1017200010F4925001C09A50923068F4803F69F0F2
:1017300018F4883E40F409C0843F29F406C0883E6E
:1017400020F0813F11F080E0089581E00895FC01D0
:10175000808191810E94770D0E948C0B0895CF9318
:10176000DF9300D000D01F92CDB7DEB70F900F905F
:101770000F900F900F90DF91CF910895CF93DF934B
:1017800000D000D000D0CDB7DEB726960FB6F894C3
:10179000DEBF0FBECDBFDF91CF91089508950895AC
:1017A0000C94CF0B0C94D00B0E94D20B6093EF01E2
:1017B0007093F0018093F1019093F2010C94700BFF
:1017C0000C94D40B0F931F930091EF011091F00133
:1017D0002091F1013091F201602B712B822B932B20
:1017E0001F910F910C94D40B0F931F930091EF0155
:1017F0001091F0012091F1013091F20160237123E9
:10180000822393231F910F910C94D40B0F931F935A
:101810000091EF011091F0012091F1013091F2015E
:1018200060277127822793271F910F910C94D40B67
:101830000C94CF0B0E94180C6093EB017093EC0199
:101840008093ED019093EE010C94700B60E070E0DA
:10185000CB010C941A0C0F931F9341E050E060E011
:1018600070E08A019B0104C0000F111F221F331F6B
:101870008A95D2F7C901B8011F910F910C941A0CE7
:101880000F931F9341E050E060E070E004C0440F0C
:10189000551F661F771F8A95D2F78091EB019091B3
:1018A000EC01A091ED01B091EE018A019B01082BA2
:1018B000192B2A2B3B2BC901B8011F910F910C94B6
:1018C0001A0C0F931F9341E050E060E070E004C0F9
:1018D000440F551F661F771F8A95D2F74095509584
:1018E000609570958091EB019091EC01A091ED01D4
:1018F000B091EE018A019B01082319232A233B237F
:10190000C901B8011F910F910C941A0C0F931F93EA
:1019100041E050E060E070E004C0440F551F661FD6
:10192000771F8A95D2F78091EB019091EC01A091FD
:10193000ED01B091EE018A019B01082719272A27A2
:101940003B27C901B8011F910F910C941A0C0F93FA
:101950001F930091EB011091EC012091ED0130916A
:10196000EE01602B712B822B932B1F910F910C9406
:101970001A0C0F931F930091EB011091EC01209131
:10198000ED013091EE0160237123822393231F9197
:101990000F910C941A0C0F931F930091EB0110916F
:1019A000EC012091ED013091EE0160277127822733
:1019B00093271F910F910C941A0C08952DE0929F7C
:1019C000800D1124E82FE695E695E695877051E0A5
:1019D00001C0550F8A95EAF785E0E89FF0011124D0
:1019E000E853FE4F20E030E070E04081CB01022E52
:1019F00002C0969587950A94E2F7817081958427B5
:101A00008523842781932F5F3F4F2530310569F768
:101A100008952DE0929F800D1124682F669566959C
:101A20006695982F977085E0689FB001112440E07B
:101A300050E080E0FB01E40FF51FE853FE4F2081EA
:101A400030E0092E02C0369527950A94E2F72170FE
:101A50003327042E01C0220F0A94EAF7822B4F5F2E
:101A60005F4F4530510531F70895BF92CF92DF9215
:101A7000EF92FF920F931F93CF93DF938C01C0904F
:101A8000EB01D090EC01E090ED01F090EE0180913F
:101A9000EF019091F001A091F101B091F201C82AFB
:101AA000D92AEA2AFB2ACFE1D0E0D701C6010C2EC1
:101AB00004C0B695A795979587950A94D2F780FDAF
:101AC00004C0219790F7B12C07C0BC2EB8018C2F11
:101AD0000E9481140197A9F38B2DDF91CF911F9163
:101AE0000F91FF90EF90DF90CF90BF900895CF932C
:101AF000DF93EC010E94350DBE010E948114DF913D
:101B0000CF9108951F93CF93DF93EB019091C7017D
:101B1000992321F0CB010E94770D13C0882349F04F
:101B2000CB010E94350D182F682FCE010E94DE0CCC
:101B300004C0CB010E94090D182FBE01812F0E9405
:101B40008114DF91CF911F9108951F93CF93DF935D
:101B5000C091F30116E08091F401C81799F0D0E02C
:101B60001C9FF0011D9FF00D1124EB50FE4F408192
:101B7000518162817381848195810E94BE0B21967F
:101B8000C770E9CFDF91CF911F9108954091250251
:101B900050912602609127027091280280912902BB
:101BA00090912A020C94BE0BEF92FF920F931F9319
:101BB000CF93DF9380912A0282958F7009F065C0E0
:101BC00080912702882309F460C08091F301F0908E
:101BD000F401109125020091260260912802709173
:101BE000290291E01F3F09F090E0C0910001D091DF
:101BF0000101292F96E0E92E8F1509F446C06115E1
:101C0000710521F00F3F21F030E003C031E001C049
:101C1000322F90E030FD36C0E89EF001E99EF00DD5
:101C20001124DF01AB50BE4F11963C911197301338
:101C300029C03C91311326C012963C911297311164
:101C400021C013964D915C911497461B570B4C176E
:101C50005D07C0F480912A028F70806180932A0210
:101C6000E650FE4F80818F708061808385E292E034
:101C70000E943C0BDF91CF911F910F91FF90EF904D
:101C80000C94A50D01968770B7CFDF91CF911F916E
:101C90000F91FF90EF9008959F92AF92BF92CF92D5
:101CA000DF92EF92FF920F931F93CF93DF93CDB705
:101CB000DEB761970FB6F894DEBF0FBECDBF8C01C3
:101CC00085E0F801DE011D9601900D928A95E1F7FD
:101CD000D8011296EC9090912502E0912602209175
:101CE0002802309129022115310531F0EF3F31F4FE
:101CF00081E09F3F19F403C081E001C080E0B82F6C
:101D0000B1709B2E80FD47C1D8014C9111965C911A
:101D100011971396AD90BC90149785E2C82E82E07F
:101D2000D82EF0902702B501621B730B20910001A1
:101D300030910101FF2009F4D9C080912A02621775
:101D4000730708F095C0282F207F09F052C05E135A
:101D500013C0491311C0FE2CE1100EC08F708061BA
:101D600080932A020E94C60DC6010E943C0B8091FE
:101D70002A02F80185834DC1AB2831F05F3F31F471
:101D800081E04F3F19F403C081E001C080E080FD95
:101D900003C081E08E2502C080E090E0F82FF17052
:101DA000FF2E80FF1CC08091F3012091F40136E0EA
:101DB000821709F40BC190E0389FF001399FF00DB4
:101DC0001124EB50FE4F6181561306C0608146130B
:101DD00003C06281E61203C001968770E9CFFE2C32
:101DE000EE2009F416C180912A02816080932A02B4
:101DF00054C05E1306C0491304C0E11002C0F801CC
:101E000099C0C8010E94A70B882361F1EE2051F10F
:101E100020912A02822F82958F7090E0029774F0B1
:101E2000809125029091260298878F831986BB8620
:101E3000AA862C87CE0107960E943C0B86E0F8010B
:101E4000A5E2B2E001900D928A95E1F70E94D40DCF
:101E50000E94C60D0AC05E1711F1C8010E94A70BAF
:101E600081112CC0C8010E943C0BFF24F394D1C007
:101E7000282F207F81F77A2DB98AA88A6E2D89892B
:101E80000E94AF0B85E292E00E943C0B86E0D601F7
:101E90001D928A95E9F70E94C60DF12CBAC049132C
:101EA000DCCFE110DACFF8018583C8010E943C0B3A
:101EB00086E0D6011D928A95E9F7ABC0EE2091F23B
:101EC00020912A02822F82958F7090E002970CF465
:101ED000B5CF80912502909126029A8389831B8237
:101EE000BD82AC822E83CE010196A6CF6217730706
:101EF00008F044C0FE2CEE2009F4B4CF5E1330C0CD
:101F000049132EC020912A0220FD21C0822F8295E4
:101F10008F70482F50E041155105C9F0F801258315
:101F20004F30510541F08F5F982F9295907F822F0F
:101F30008F70892B8583C8010E943C0B86E0F801D5
:101F4000A5E2B2E001900D928A95E1F73CC086E0EF
:101F5000F801A5E2B2E001900D928A95E1F759C02F
:101F6000C8010E94A70B811169CF80912A0281606C
:101F700080932A02C8010E943C0B4BC07A2DB98A7B
:101F8000A88A6E2D89890E94AF0B86E0D6011D922A
:101F90008A95E9F718C0EE2009F464CFC8010E94C1
:101FA000A70BF82E882309F45DCF86E0F801A5E29F
:101FB000B2E001900D928A95E1F785E292E00E94ED
:101FC000A8070E94D40D0E94C60D23C04D875E87CE
:101FD0008D859E850E94770D292F22952F702230A6
:101FE00028F49F7039F0811105C00BC0243028F40B
:101FF0009F7049F4805E883020F0C8010E943C0B3D
:102000009F2CF92C06C0D80115969C91907F91F7D2
:10201000F8CF8F2D61960FB6F894DEBF0FBECDBFFF
:10202000DF91CF911F910F91FF90EF90DF90CF90B4
:10203000BF90AF909F9008951F93CF93DF93CDB73C
:10204000DEB72C970FB6F894DEBF0FBECDBF4F831F
:10205000588769877A878B879C87CE0107960E946D
:102060004C0E8823D1F09F8188852A853B85232BC0
:1020700031F08F3F31F481E09F3F19F403C081E0DC
:1020800001C080E080FD47C04F81588569857A8511
:102090008B859C850E94BE0B3EC086E0FE01379674
:1020A000DE01119601900D928A95E1F7FF81E88596
:1020B0006A857B856115710531F0EF3F31F481E070
:1020C000FF3F19F403C081E001C080E080FD23C020
:1020D0002091F40130E0C901019687709927409161
:1020E000F30150E084179507F1F1F983EA837D83CA
:1020F0006C8396E0929FD001939FB00D1124AB505A
:10210000BE4FFE01319601900D929A95E1F78093B2
:10211000F4010E94A50D16E08091F3019091F40165
:10212000891771F1189FC00111248B509E4F0E9496
:102130004C0E882329F1E091F3011E9FF001112438
:10214000EB50FE4F40815181628173818481958182
:102150000E94BE0B8091F30190E001968770992751
:102160008093F301D9CF0E94880B1092F401109252
:10217000F301E5E2F2E086E0DF011D928A95E9F7DE
:102180002C960FB6F894DEBF0FBECDBFDF91CF9176
:102190001F910895809133028595859585950895C1
:1021A000809133028770089590913302977081E097
:1021B00009F480E0089580913E02089590913E02D6
:1021C000892B80933E020895809590913E02892349
:1021D00080933E02089510923E02089590913D0230
:1021E000892B80933D020895809590913D0289232B
:1021F00080933D02089510923D020895809134022B
:10220000089508950C9401110C94021190918A0282
:1022100092FD08C090913402981721F08093340207
:102220000C940411089580913402882329F01092AF
:10223000340280E00C9404110895CF93DF93E09171
:102240000201F091030180913E028083E09102013E
:10225000F0910301908180913D02892B80838091D0
:102260003402882381F0E0910201F0910301908112
:10227000892B808380910201909103010E94BA24EE
:1022800081110E941311C0910201D091030148E015
:1022900050E06BE272E0CE010E94752D892B69F04F
:1022A00088E0FE01ABE2B2E001900D928A95E1F781
:1022B000CE01DF91CF910C947524DF91CF910895D9
:1022C0000C94011190918A0292FD10C098E0899FB0
:1022D00090011124262B209333020E94400C809100
:1022E00033028595859585950C9460110C94400C6E
:1022F0001092330280E00C9460112091330280959B
:10230000822380933302982F977099F430E0482FFE
:10231000082E000C550B2417350759F090918A02AE
:1023200092FD07C08595859585950E94610C0C945A
:102330007811089590918A0292FB222720F928179C
:1023400069F080FB92F990938A02809189029091C2
:102350008A020E94E71182E00C947D110895809119
:102360008A0282FB882780F991E089270C949A11D0
:1023700081E00C949A1180E00C949A1180E090E036
:102380000E94902D21E0893E9E4F09F020E0822F8F
:10239000089582E090E00C94822D83E090E00C940C
:1023A000822D682F83E090E00C94962DCF9384E0EB
:1023B00090E00E94822DC82F82E290E00E94822D40
:1023C0002C2F30E0A901582BCA01CF910895CF934B
:1023D000C92F682F84E090E00E94962D6C2F82E236
:1023E00090E0CF910C94962DAB01BC018FE090E072
:1023F0000C94A82DAB01BC0183E190E00C94A82DB6
:1024000060E070E0CB010C94FA1160E070E0CB0169
:102410000E94F4110C94001269EE7EEF80E090E0CF
:102420000E94B42D60E082E090E00E94962D60E072
:1024300083E090E00E94962D1092EF011092F0013F
:102440001092F1011092F20160E084E090E00E94AD
:10245000962D60E082E290E00E94962D60E085E09B
:1024600090E00E94962D60E086E090E00E94962D1C
:102470006FEF87E090E00E94962D40E050E0BA01B7
:1024800088E090E00E94A82D60E08DE090E00E943E
:10249000962D40E050E0BA0188E190E00E94A82D1E
:1024A00060E087E190E00E94962D40E050E0BA01A4
:1024B0008CE190E00E94A82D60E070E080E290E066
:1024C0000E94B42D40E050E0BA0188E190E00E9403
:1024D000A82D0C9405120C940C12682F8EE090E03D
:1024E0000C94962D0E94AF2560934B0270934C0282
:1024F00080934D0290934E0260934702709348027E
:102500008093490290934A02089585B7806885BFF9
:1025100085B7806885BF089581E008950C948C127A
:1025200008950C9490120C9490120C9493120C94A5
:1025300090120C9497120C9490120E9485128DE5C3
:1025400095E10E945F240E949B120C9499120E94B4
:1025500091120C9490120E9460150C9442070E94F4
:102560009A250E9441160E94AB120E94CF1E0C9425
:1025700095125F926F927F928F929F92AF92BF92CD
:10258000CF92DF92EF92FF920F931F93CF93DF933F
:10259000CDB7DEB72A970FB6F894DEBF0FBECDBF1A
:1025A0000E945616C82E81110E9472123FE3832E9C
:1025B00032E0932E00E010E0502E802F0E94841510
:1025C0005C01F401619071904F01682679266114D5
:1025D0007104B1F40F5F1F4F0430110569F78FEFDD
:1025E00089838A831B820E94A3258160782F9D8323
:1025F0008C8349815A816B818D810E945E073AC02C
:1026000080914F0281FD0E948D15D12CEE24E39420
:10261000F12CC3018E219F21892B29F10E948E125A
:102620008823A9F0DE825F82AE20BF2081E0AB2844
:1026300009F480E088870E94A3258160782F9A871B
:1026400089874E815F8168858A850E945E07000FB9
:10265000111FF801E15CFD4F80819181E826F92688
:10266000F182E08207C0D394EE0CFF1CFDE0DF1284
:10267000D0CFB0CF81E0C11001C080E02A960FB664
:10268000F894DEBF0FBECDBFDF91CF911F910F91A8
:10269000FF90EF90DF90CF90BF90AF909F908F9082
:1026A0007F906F905F9008950E94B9120E94021F60
:1026B0000E945D180C945307CF93DF930E948614F9
:1026C000EC01811521E5920708F045C0811530E540
:1026D000930708F094C0883E910528F5803E910547
:1026E00008F0F8C0883A910570F4853A910508F031
:1026F0007CC08130910509F475C008F4E8C00497E6
:1027000008F0E8C0E4C08F3B910508F0E0C0C85A6B
:10271000D0E0CC0FDD1FC35ADE4F0990D881C02D09
:10272000CE019464D8C0811540E2940758F4811515
:1027300051E0950708F0CEC08D3E910508F4C7C062
:102740009065C9C0C11580E4D80708F4C0C0DF7027
:10275000CE01906AC0C0811525E59207A8F48115C5
:1027600034E5930708F095C0811543E5940708F018
:102770007BC0811552E5950708F061C0D82FCC27A2
:10278000CE01816F906AA7C0C11589E5D807A0F472
:10279000C11528E5D20708F082C0C11536E5D30778
:1027A00008F095C08C2F0E941A158F7190E0D82FD9
:1027B000CC27CE0190628FC0C1154AE5D40708F43A
:1027C00074C0CE0190568115904208F080C08D2FC4
:1027D0008F710E941A15DD27D0628F71AE01582BC0
:1027E000CA0179C081E090E076C0C55AD0E0C557F3
:1027F000DE4F8881C82FD0E0CE0190646CC074E0B9
:10280000969587957A95E1F7282F23703C2F3370A2
:1028100081E090E002C0880F991F3A95E2F79C682A
:10282000AC01522B9A019C2F9F709695969550E281
:10283000959FE0011124C9018C2B9D2B4CC0837006
:10284000992721E030E002C0220F331F8A95E2F77A
:102850009C2F9695969580E2989FE0011124C22BBB
:10286000D32BCE019C6837C08370992721E030E0DC
:1028700002C0220F331F8A95E2F79C2F96959695FA
:1028800040E2949FE0011124C22BD32BCE019A6821
:1028900022C0D82FCC27CE01846F906A1CC0DC2FB9
:1028A000CC27CE01806F906A16C08C2F8F700E944B
:1028B0001A1594E0D695C7959A95E1F7CF70D0E0B8
:1028C000DC2FCC27D0699E01282BC90104C080E0F1
:1028D00090E001C0CE01DF91CF91089524E3829F63
:1028E000C0011124FC012DE0729FE00DF11D1124A7
:1028F000E60FF11DEE0FFF1FE852FF4F85919491F7
:1029000008950E946E140E945C1308958238910508
:1029100069F1B0F48133910509F46DC048F489324E
:10292000910509F463C08A32910509F469C00895DC
:102930008533910509F455C089339105B9F008959F
:10294000833E910569F138F4803E9105B1F0823EF5
:10295000910509F10895863E9105A9F1873E9105FB
:10296000B9F1843E910509F064C023C02091890229
:1029700020FD4FC021FD4DC008958091890280FD4A
:1029800044C080918A0280FF44C08091890284FD06
:1029900042C083EE4DC08091890282FF38C0F5CFDE
:1029A0008091890282FD33C080918A0280FD31C00E
:1029B000ECCF80918A0281FF32C08091890284FD30
:1029C0002AC087EE35C08091890283FF26C0F5CFEB
:1029D0008091890283FD21C080918A0281FD1FC000
:1029E000ECCF8091890285FD1CC01DC080918902B9
:1029F00085FD19C016C08091890286FD16C017C0DA
:102A00008091890286FD13C010C089E311C082EE57
:102A10000FC080EE0DC080E00BC086EE09C084EED2
:102A200007C089E205C085E303C08AE201C081E3F3
:102A300090E008959091890292FF0DC0282F28718F
:102A4000283019F4877F846006C0282F2471243031
:102A500011F48B7F886093FF0DC0282F28712831D7
:102A600019F4877E846106C0282F2471243111F463
:102A70008B7E886120918A0220FF0DC0382F38712B
:102A8000383019F4877F816006C0382F31713130BA
:102A900011F48E7F886021FF0DC0282F2871283106
:102AA00019F4877E816106C0282F2171213111F42C
:102AB0008E7E886194FD877E089580E00895089554
:102AC0000E94BE11811102C00E946B120E94C911A6
:102AD00080934F020E94D61190938A0280938902BC
:102AE0000E945F150E94CD11682F70E080E090E099
:102AF0000E94E00B6091EB017091EC018091ED017F
:102B00009091EE010C94180CE82FF0E0EE0FFF1FEF
:102B1000ED56FD4F808191810895089580EA8A9550
:102B2000F1F7089500C008950C948E1508950C9443
:102B300096150C949715F894E82FE295EF70F0E055
:102B400031A1282F2F7081E090E001C0880F2A95D5
:102B5000EAF7982F9095932391A392A1892B82A3B2
:102B6000789408950F931F93CF93DF93CBE9D1E02F
:102B700089918F3F11F00E949B1581E0CF39D807D2
:102B8000B9F7CEE8D1E00BE911E089918F3F11F060
:102B90000E949B150C171D07C1F7DF91CF911F9164
:102BA0000F910895BF92CF92DF92EF92FF920F9311
:102BB0001F93CF93DF938C01C62FD0E0CE018556B3
:102BC0009E4F6C01FC0190819F3F09F450C0B62ECE
:102BD000F894E92FE295EF70F0E081A19F7021E079
:102BE00030E001C0220F9A95EAF7822B81A382A1DF
:102BF0002095282322A378940E949215EEE8F1E014
:102C00004BE951E021E030E0E12CF12C61916F3F84
:102C100089F0A62FA295AF70B0E090968C9190E0CD
:102C20006F7002C0959587956A95E2F780FD02C0A6
:102C3000C90102C080E090E0E82AF92A220F331F80
:102C40004E175F0719F7F60180818F3F11F00E9440
:102C50009B1561E0E114F10409F460E08B2D0E9402
:102C60009415CC0FDD1FC00FD11FF982E882DF91D0
:102C7000CF911F910F91FF90EF90DF90CF90BF9079
:102C800008950E94B21588E0E3E9F2E0DF01982F91
:102C90001D929A95E9F7EBE8F2E0DF011D928A9523
:102CA000E9F784E00E94A1160C94C606FF920F93E8
:102CB0001F93CF93DF93CDB7DEB728970FB6F89465
:102CC000DEBF0FBECDBF8E010F5F1F4F88E0F80142
:102CD00011928A95E9F7F12C6F2DC8010E94D21547
:102CE000F394F4E0FF12F8CF48E050E0B8018BE82D
:102CF00092E00E94752DFF24F394009709F4F12CC3
:102D0000892B41F088E0F801ABE8B2E001900D9228
:102D10008A95E1F72F2D44E063E972E08BE892E0B9
:102D20000E94A2160E94C8068F2D28960FB6F8940E
:102D3000DEBF0FBECDBFDF91CF911F910F91FF90EE
:102D400008950895FF920F931F93CF93DF93F82E6A
:102D5000092F162FD72FC42F222349F081E080930B
:102D600052020E94A32590935102809350028091B9
:102D700052028823D9F080915002909151020E9412
:102D8000BB25059798F0EF2DF02FA12FBD2F80E0E8
:102D900090E04C2F50E08417950734F42191319145
:102DA0002D933D930196F7CF10925202DF91CF9170
:102DB0001F910F91FF9008950E9493270E94AF12D8
:102DC0000C949F270E94A3270E9454130C94BD27A4
:102DD0000E9441250E947A270E949D120E94DC16C3
:102DE0000E94E2160E94A712FBCF8091590280FF39
:102DF00006C06091090170E0660F771F26C081FF51
:102E000004C06091090184E005C082FF07C06091A1
:102E1000090188E0689FB001112417C09091580201
:102E20009923D1F060910801961788F72091090144
:102E300088E0289F90011124929FA001939F500D3C
:102E4000112470E0CA010E94EF2C6038710540F433
:102E50006115710519F406C068E070E0862F0895C9
:102E60008FE7089581E008958091590280FF08C09E
:102E70006091050170E0759567957595679521C01E
:102E800081FF06C06091050170E07595679519C0D6
:102E900082FF04C06091050170E010C0909157025C
:102EA000992399F0609104019617A0F7809105018C
:102EB000899FC001112470E00E94EF2C60387105D9
:102EC00040F46115710519F406C061E070E0862FC9
:102ED00008958FE7089581E008958D3E21F40E94C2
:102EE000F516819504C08E3E29F40E94F516809354
:102EF0005D0208958F3E21F40E94F516819504C06D
:102F0000803F29F40E94F51680935C020895893F62
:102F100019F40E94341705C08A3F31F40E94341717
:102F2000819580935E0208958B3F21F40E943417AF
:102F3000819504C08C3F29F40E94341780935F026E
:102F400008959FE0980F983078F421E030E0A901CF
:102F500002C0440F551F9A95E2F7CA0190915B0297
:102F6000892B80935B0208958D3F21F48091590253
:102F700081600BC08E3F21F480915902826005C0B0
:102F80008F3F29F4809159028460809359020895FB
:102F90008D3E39F490915D0297FF35C010925D022D
:102FA00059C08E3E29F490915D021916BCF32BC0D6
:102FB00090915C028F3E29F497FF25C010925C022D
:102FC00049C0803F19F41916CCF31DC090915E02E0
:102FD000893F29F41916BCF410925E023BC08A3F67
:102FE00019F497FF10C0F8CF8B3F39F490915F022E
:102FF00097FF09C010925F022DC08C3F21F4909181
:103000005F021916BCF39FE0980F983080F421E01E
:1030100030E0A90102C0440F551F9A95E2F7CA019A
:10302000809590915B02892380935B0213C08D3F52
:1030300021F4809159028E7F0BC08E3F21F4809144
:1030400059028D7F05C08F3F29F4809159028B7FF3
:103050008093590280915C02811106C080915D02CB
:10306000811102C01092580280915E02811106C047
:1030700080915F02811102C01092570208950E9450
:10308000A32520915C02211104C020915D0222231E
:1030900021F0909356028093550220915E022111F7
:1030A00004C020915F02222321F090935402809368
:1030B00053028AE592E00C948024EF92FF920F93E2
:1030C0001F93CF93DF9300D000D000D0CDB7DEB7F1
:1030D00086E0EAE5F2E0DE01119601900D928A9514
:1030E000E1F7E0905C02F0905D0200915E021091C9
:1030F0005F0210925C0210925D0210925E021092CA
:103100005F02E11003C0FF2009F45DC08091550209
:10311000909156020E94BB25AC01909158029923D0
:1031200039F020910A0130E02417350758F04BC0E0
:1031300020910B018AE0289F900111242417350764
:1031400018F041C09F3F19F09F5F90935802EE2006
:1031500061F00E94F5161E1414F09FEF01C091E07B
:10316000989F902D112490935C02FF2061F00E94A3
:10317000F5161F1414F09FEF01C091E0989F902D59
:10318000112490935D0230915C023323E1F0209191
:103190005D022223C1F045EB3403C00111249923C1
:1031A00019F090935C0203C081E080935C0235EBE0
:1031B0002303C0011124992319F090935D0203C0E9
:1031C00081E080935D02011103C0112309F45DC009
:1031D00080915302909154020E94BB25AC019091C2
:1031E0005702992339F02091060130E02417350762
:1031F00058F04BC0209107018AE0289F90011124CC
:103200002417350718F041C09F3F19F09F5F909336
:103210005702002361F00E943417101614F09FEF3C
:1032200001C091E0989F902D112490935E0211238C
:1032300061F00E943417111614F09FEF01C091E065
:10324000989F902D112490935F0230915E0233235A
:10325000E1F020915F022223C1F045EB3403C0016D
:103260001124992319F090935E0203C081E08093AA
:103270005E0235EB2303C0011124992319F09093CA
:103280005F0203C081E080935F0280915C02811144
:103290000BC080915D02811107C080915E02811197
:1032A00003C080915F0281110E943F18EB82FC8273
:1032B0000D831E8386E0FE013196AAE5B2E00190FF
:1032C0000D928A95E1F726960FB6F894DEBF0FBEF1
:1032D000CDBFDF91CF911F910F91FF90EF90089597
:1032E000EAE5F2E086E0DF011D928A95E9F71092A7
:1032F000580210925702109259020895EF92FF92CD
:103300000F931F93CF93DF938B01682F11110AC086
:10331000442329F0E82FF0E0E952F74F6491762F2B
:10332000862F75C0212F30E0E82FF0E0442321F0F4
:10333000E952F74FE491F0E046E0049FC001112408
:10334000CFEFD0E0BE010E94DB2C4BEA4603C00168
:10335000479F900D1124800F911D800F911D982F74
:10336000990F890FAE01421B530B4E9FD0014F9F07
:10337000B00D5E9FB00D11249B2F189FA00111244A
:10338000452F55278E01041B150B0E9FA0010F9F83
:10339000500D1E9F500D11247E01E81AF108E29E87
:1033A0008001E39E100DF29E100D1124212F332772
:1033B000C21BD30BCE9F9001CF9F300DDE9F300DEF
:1033C000112462307105A9F048F46115710569F0A6
:1033D00061307105C9F48B2F752F0DC064307105F4
:1033E00081F058F06630710579F47E2F8B2F932F82
:1033F0000DC0832F7B2F9E2F09C08E2F7B2F952FE3
:1034000005C08E2F732F02C07E2F852F692FDF916D
:10341000CF911F910F91FF90EF90089541E00E948E
:103420007E19089508950E940E1A0895CF93DF9390
:10343000762FE901682F842F0E94131A79836883FD
:103440008A83DF91CF91089580919B02282F269542
:1034500030E02115310519F48170826005C02532F4
:10346000310524F08170886480939B02089588E080
:1034700090E00C948A2DCF92DF92EF92FF926B0135
:103480007C010E94241AB701A60188E090E0FF9019
:10349000EF90DF90CF900C94A82DEBE9F2E083E061
:1034A000808311828FEF8283838314826081718194
:1034B000828193810C943B1A80919B0280FF02C011
:1034C0008695089580E0089590919F02933018F4B6
:1034D0009F5F90939F02882351F060919B027091AF
:1034E0009C0280919D0290919E020C943B1A08953B
:1034F00081E00C94641A90919F02992319F09150E5
:1035000090939F02882351F060919B0270919C02DE
:1035100080919D0290919E020C943B1A089581E047
:103520000C947B1A70E00C947F20609110018091C4
:103530009B0280FF0AC080910F0123E0829FC0019F
:10354000112480569D4F0C94921A809111019091F4
:103550001201891780F7E82FF0E09F01220F331F37
:10356000E20FF31FE056FD4F1182108212828F5F2F
:10357000F0CF90919B0290FF16C090911101209185
:103580001201921770F4E92FF0E0DF01AA0FBB1FC0
:10359000EA0FFB1FE056FD4F8183608342839F5FEC
:1035A000F0CF0C94951A0895CF93DF9300D01F921B
:1035B000CDB7DEB790919B0290FF0AC09E012F5FAE
:1035C0003F4F0E94161A4B8169818A810E94B91A65
:1035D0000F900F900F90DF91CF910895CF93DF93CD
:1035E000EC01EC81F0E0EE52F84F4491EBE9F2E0AF
:1035F000628181810E94D41A8C818F5F8C83DF91DC
:10360000CF910895CF93DF93EC01EBE9F2E0438192
:1036100062818C810E94D41A8C818F5F8C83DF91B0
:10362000CF9108950F931F93CF93DF9300D01F92F4
:10363000CDB7DEB78C018091600281110AC09E0176
:103640002F5F3F4F4FEF6FEF0E94161A8A818093D2
:103650006002F8018481813051F028F0823061F4F9
:10366000409160020AC08091600240E007C0609112
:10367000600240E080E003C040E080E060E00E9443
:10368000B91AF801848190E0019663E070E00E942D
:10369000EF2C84830F900F900F90DF91CF911F91AB
:1036A0000F910895AF92BF92CF92DF92EF92FF9267
:1036B0000F931F93CF93DF9300D01F92CDB7DEB748
:1036C000182FF62E042FE22E90919B0290FF6DC0D2
:1036D000E92FE695AE2FB0E0A156BE4F8C918093B6
:1036E0006A029E7F923061F49E012F5F3F4F812FCF
:1036F0000E94161A4B8169818A810E94B91A43C0BF
:10370000823019F400919E023EC0863019F4109167
:103710009C0239C08930D9F38931A9F5E9518E2F3E
:103720008170D82EE695F0E0EE52F74FA590B49058
:10373000C12CBB2460911301C61618F52C2D30E066
:10374000A29EC001A39E900DB29E900D112470E028
:103750000E94DB2C812FD11002C0860F01C0861B76
:1037600090911101290F311DA901440F551F240FFC
:10377000351F20563D4F402F6F2D0E94161AC394BF
:10378000D9CF0E94951A10939C02F0929D0200934B
:103790009E02EE2051F060919B0270919C028091FC
:1037A0009D0290919E020E943B1A0F900F900F90E5
:1037B000DF91CF911F910F91FF90EF90DF90CF900D
:1037C000BF90AF900895EBE9F2E09181282F4381FB
:1037D00062818AE0890F0C94521B81E00C94E31BF8
:1037E000EBE9F2E09181282F4381628186EF890F16
:1037F0000C94521B81E00C94F01BEBE9F2E0628127
:1038000021E1620F08F46FEF282F438181810C942E
:10381000521B81E00C94FD1BEBE9F2E0628121E197
:10382000621B08F460E0282F438181810C94521BB5
:1038300081E00C940C1CEBE9F2E0438121E1420FA2
:1038400008F44FEF282F628181810C94521B81E094
:103850000C941B1CEBE9F2E0438121E1421B08F4CC
:1038600040E0282F628181810C94521B81E00C94EE
:103870002A1C20E00C94521BFF920F931F93CF93AE
:10388000DF93EC01F12C0FEF10E060911301F616BD
:10389000F0F4809111012F2D30E0280F311DC90166
:1038A000880F991F280F391F20563D4F70E0C8011F
:1038B0000E94EF2C962F8C8140919E0260919D0278
:1038C000F99E800D11240E94161AF394DECF0E94F7
:1038D000951A9A818C8190FF02C08F5F01C0815040
:1038E0008C83DF91CF911F910F91FF900895AF923C
:1038F000BF92CF92DF92EF92FF920F931F93CF93DD
:10390000DF93FC01828180FF02C00FEF01C001E064
:1039100010E04CE0A42E80911301181708F043C06A
:1039200080911101C12ED12CE601C80FD11DCE010D
:10393000880F991FC80FD91FC056DD4F19821882F2
:103940001A8234E0E32EF12CB12C809162028B0DAF
:103950008D302CF06A2D0E94CD2C892F05C087FF59
:1039600003C090911301890F082E000C990BC81603
:10397000D90691F480919E028E9DA0018F9D500DDD
:10398000112455954795559547959E0160919D0247
:1039900080919C020E94161AB00EF1E0EF1AF10815
:1039A000A1F61F5FB8CF0E94951A80916202013084
:1039B00031F4811102C080911301815007C090E061
:1039C00001966091130170E00E94EF2C80936202D7
:1039D000DF91CF911F910F91FF90EF90DF90CF90EB
:1039E000BF90AF900895CF938091110190911201F3
:1039F000891770F4E82FF0E09F01220F331FE20FC8
:103A0000F31FE056FD4F1182108212828F5FF0CFBC
:103A1000C0E060911301C617C0F5EC2FF0E070E034
:103A2000CF010E94EF2C20911101820F20916102A1
:103A3000022E000C330B90E0E217F307CCF020913C
:103A40000E01022E000C330B2E173F078CF09C0149
:103A5000220F331F820F931F9C0120563D4F409130
:103A60009E0260919D0280919C020E94161A0BC0DA
:103A7000FC01EE0FFF1F8E0F9F1FFC01E056FD4F54
:103A8000118210821282CF5FC4CF0E94951A2091BA
:103A90000D0180916102820F8093610290910E016D
:103AA000920F90930E0119165CF4082E000C990BDE
:103AB0004091130150E041505109841795071CF0C3
:103AC000219520930D01CF9108958F929F92AF92EF
:103AD000BF92CF92DF92EF92FF920F931F93CF93FB
:103AE000DF938C01FC014481C42FD0E09E01DE01F4
:103AF0000E94332D9B01AC010E94492D6B017C017A
:103B0000E0E2F0E0EC1BFD0BA5E5B0E09B01AC01B1
:103B10000E94492D4B015C019F01DF010E942B2D6A
:103B20009B01AC010E94542D9B01AC012C0D3D1D4D
:103B30004E1D5F1DC501B4010E94032DC22FD22F5F
:103B40002A3228F4F3E02F9F900111240DC025E5BF
:103B500030E02C1B3109C901880F991F280F391F2C
:103B600037FF02C02F5F3F4F35952795C22FC09575
:103B7000F12C85E5E82EED1A80911301F816C8F4B2
:103B8000F1FC02C08E2D01C08D2F909111012F2DBF
:103B900030E0290F311DA901440F551F240F351F97
:103BA00020563D4F4C2F60919D020E94161AF394AF
:103BB000E3CF0E94951AF8018481811102C091E03F
:103BC00003C0803219F49FEF90930C0190910C0187
:103BD000890FF8018483DF91CF911F910F91FF909E
:103BE000EF90DF90CF90BF90AF909F908F9008950F
:103BF0000F931F93CF93DF93EC0100E010E08091CF
:103C00001301282F30E00217130724F590911101BA
:103C10009801290F311DA901440F551F240F351F8D
:103C200020563D4F869590E04C81081719071CF4EB
:103C3000442331F002C0411103C040919E0201C0F3
:103C400040E060919D0280919C020E94161A0F5FD5
:103C50001F4FD5CF0E94951A8C8190E001968170FC
:103C600099278C83DF91CF911F910F910895EBE9F4
:103C7000F2E080818E7F8083608171818281938177
:103C80000E943B1A10926B022FEF80E792E02150C6
:103C900080409040E1F700C000000C94951A6091BC
:103CA0009B02669570E04BE050E084E191E00E9459
:103CB000682D892B19F481E080936B020E94A32563
:103CC0009093640280936302089590919B0290FF09
:103CD00035C09170811102C0926006C0853210F02B
:103CE000986402C0880F982B90939B02662351F032
:103CF00060919B0270919C0280919D0290919E0226
:103D00000E943B1A60919B02669570E04BE050E088
:103D100084E191E00E94682D892B19F010926B02CA
:103D200002C00E944F1E81E08093660240919E0275
:103D300060919D0280919C020C94391C0895682F1B
:103D400090919B02969581E0890F853208F081E081
:103D50000C94651E81E00C949F1E682F90919B022D
:103D600096958FEF890F09F484E20C94651E81E02B
:103D70000C94AD1E61E00C94651EEBE9F2E08081CD
:103D80008160808386950C94BA1E80919B0280FD91
:103D90000C94371E0C94BD1E60E00C94651E80913F
:103DA000690281112EC00E94BE11811104C00E94BF
:103DB0006B120E944D1A0E94371A60939B027093F7
:103DC0009C0280939D0290939E026E7F61F40E94FC
:103DD0004D1A0E94371A60939B0270939C02809345
:103DE0009D0290939E020E94241A10926B02809171
:103DF0009B0280FF03C086950E94CC1E81E08093C9
:103E0000690208950F931F93CF93DF9380916B0204
:103E1000882309F485C080916A02E0919B02E695AF
:103E2000E81BE0936502823049F4F0E0E253F84F7A
:103E3000E491CE2FD0E00EEE1AE149C0863049F46D
:103E4000F0E0E553F84FE491CE2FD0E002E01BE123
:103E50003EC0893051F4E695F0E0E853F84FE49124
:103E6000CE2FD0E00CE31CE132C08F3051F4E69548
:103E7000F0E0EB53F84FE491CE2FD0E007E71CE1E0
:103E800026C0853149F4F0E0EE53F84FE491CE2F8F
:103E9000D0E003EF1CE11BC0883181F0833239F49C
:103EA000E0ECF7E0C591D49102E11BE110C084324F
:103EB00051F4C4EFD1E008EF1DE109C0C8E2D0E041
:103EC00005E61DE104C0C0EDD7E002E11AE18091F2
:103ED0006602882361F0109266020E94A3259093E7
:103EE00064028093630210926802109267020E943B
:103EF000A325E0916302F09164028E1B9F0B8F3F1C
:103F00009F4770F4EC0FFD1FF0936402E09363028F
:103F100083E692E0F801DF91CF911F910F91099410
:103F2000DF91CF911F910F910895882311F0FA012D
:103F300001C0FB010994CF93DF93C82FD62F0E94B5
:103F40005C1A8C1740F00E945C1A8D1720F4DF91E8
:103F5000CF910C94AA1E8C2FDF91CF910C94BA1E96
:103F60001F93CF93DF93FB0112811111C3C0EC01AA
:103F70000E94DB108272CD3CFCE5DF0709F49AC099
:103F8000A8F5C73CECE5DE0709F476C0A8F4C43C0C
:103F90009CE5D90709F45FC028F4C33CDC4509F46B
:103FA00057C054C0C53C9CE5D90709F459C0C63C6C
:103FB000DC4509F45CC04AC0CA3CFCE5DF0709F4F3
:103FC0006AC050F4C83CECE5DE0709F45AC0C93CAD
:103FD000DC4509F45BC03AC0CB3C9CE5D90709F449
:103FE0005FC0CC3CDC4509F460C030C0C23DFCE59C
:103FF000DF0709F46FC088F4CF3C9CE5D90709F4CA
:1040000060C008F45CC0C03DFCE5DF0709F45CC09B
:10401000C13DDC4509F45BC019C0C53D9CE5D9072D
:1040200009F460C050F4C33DFCE5DF0709F455C056
:10403000C43DDC4509F454C009C0C63D9CE5D90720
:1040400009F455C0CE35DD4509F454C011E052C025
:104050000E94C51E4FC047EB5EE16AEA7EE104C0E4
:104060004AEA5EE167EB7EE10E94951F43C04AEF9A
:104070005BE16DEE7BE1F8CF4DEE5BE16AEF7BE15A
:10408000F3CF48E15CE169E07CE1EECF49E05CE13F
:1040900068E17CE1E9CF46E35CE167E27CE1E4CF03
:1040A00047E25CE166E37CE1DFCF4FE85AE168E795
:1040B0007AE1DACF48E75AE16FE87AE1D5CF81E0DB
:1040C00017C065E082E010C068E086E00DC06EE0D9
:1040D00089E00AC064E18FE007C067E185E104C0C0
:1040E00088E106C062E289E10E949B1F03C083E26F
:1040F0000E94BA1E812FDF91CF911F9108953E9AA1
:1041000028B12F7B38B130644FB7F894FC01CB0154
:10411000880F991F680F791F6E0F7F1FE617F7072B
:1041200089F0819198E038B9000000C087FF28B974
:10413000880F000000C000C000C028B900C09A95D8
:1041400091F7ECCF4FBF8FE594E00197F1F700C0F6
:1041500000000895CF93DF93EC01FB018281882357
:1041600009F43CC1C430FDE5DF0760F4CB3F9CE5BA
:10417000D90788F49E0122503C452431310508F0CE
:104180002EC109C0C236EDE5DE0729F0C63AFDE5CD
:10419000DF0709F024C10E94D61190938A02809310
:1041A0008902C1318CE5D80709F4C6C008F042C0C5
:1041B000C930ECE5DE0709F49BC000F5C5308CE59D
:1041C000D80709F485C078F4C330ECE5DE0709F4BC
:1041D00078C008F07AC0C230DC4509F0F5C08091A3
:1041E00089028160EFC0C7309CE5D90709F478C027
:1041F00008F07AC0809189028061E4C0CD30FCE58E
:10420000DF0709F487C058F4CB309CE5D90709F4DF
:1042100079C008F07BC08091890288606FC0CF3080
:10422000FCE5DF0709F480C008F082C080918902B4
:10423000877FC8C0CE3F9CE5D90709F471C000F55F
:10424000C531FCE5DF0709F485C068F4C3319CE59E
:10425000D90709F475C008F095C00E94880B8091B9
:1042600089028F77AFC0CC3FFCE5DF07A9F108F0EA
:1042700054C0CB3FDC4509F0A7C080918A0240C002
:10428000C230EDE5DE0709F489C058F4C1158DE5AB
:10429000D80709F45AC008F069C080918A02826088
:1042A0002FC0C236EDE5DE0709F47CC0C63AFDE555
:1042B000DF0709F481C0C330DD4509F085C080E027
:1042C0006EC08091890282607DC08091890216C093
:1042D00080918902886076C080918A0282604FC096
:1042E0008091890280626EC08091890280646AC078
:1042F0000E94880B80918902806864C0846062C0DB
:1043000081603DC0809189028E7F5CC0809189026E
:104310008D7F58C08091890216C080918A0218C092
:1043200080918A028D7F2BC0809189028F7E4AC046
:10433000809189028F7D46C0809189028F7B42C027
:1043400080918902877F8B7F3DC080918A028D7F1B
:104350008E7F15C08091890282FB222720F991E08F
:10436000922790FB82F990FB83F92CC080918A02FE
:10437000982F909591708E7F892B90FB81F9809377
:104380008A0222C00E94880B8091890287FB222723
:1043900020F991E0922790FB87F914C081E00E94F8
:1043A0006D1212C08091890284FB222720F991E0CE
:1043B000922790FB84F906C080918902982F9095EE
:1043C00090FB80F9809389028091890290918A0202
:1043D0000E94E7110E94880B80E001C081E0DF911C
:1043E000CF910895893289F1F0F4843171F1B0F4FC
:1043F000873009F077C081E080930B0184E18093DE
:104400000A018AE0809309018EE18093080188E027
:104410008093050188E28093040164C092EE980FB6
:104420009A30F0F05FC0803509F444C028F48F342E
:1044300009F058C08AE03FC0813529F0823509F083
:1044400051C081E038C08FEF36C080916E02882362
:1044500079F110926E0210926D0210926C0242C0BD
:104460008D5180936E02833099F038F4813069F079
:104470008230D9F48AE091E00DC0853099F078F06F
:10448000863099F484E091E005C08BE091E002C0B1
:1044900089E091E090936D0280936C0223C088E0E4
:1044A00091E0F8CF85E091E0F5CF10926E021AC04E
:1044B00080E0089586EFE0916C02F0916D023097F4
:1044C00089F02081082E000C990B820F911D8F3FDF
:1044D000910519F014F08FEF04C097FF02C010820D
:1044E00001C0808381E008950F931F9341E050E065
:1044F00060E070E08A019B0104C0000F111F221FC1
:10450000331F8A95D2F7C901B8010E94E00B1F91B1
:104510000F910C94880B8B3109F468C058F58B30DF
:1045200009F486C078F4863009F445C020F485305B
:1045300009F44BC07FC0873009F44AC0883009F4C1
:1045400077C078C0803109F464C068F48E3009F017
:1045500071C080914F0282FB222720F991E09227BF
:1045600090FB82F94CC0863109F462C0893109F4AC
:104570005FC060C08A32E1F060F4873209F455C050
:1045800028F48E3108F456C08D5150C08932E9F0BC
:1045900051C0833450F48A3308F045C0853309F4A0
:1045A00044C0883309F444C045C08334F1F142C0AB
:1045B0000E946B123DC080914F02817F8E7F80935D
:1045C0004F0281E080936F0208950E94CB0630C0B5
:1045D00080914F02982F9095917090FB80F9809375
:1045E0004F02911125C0897F877F10C080914F02B3
:1045F00081FB222720F991E0922790FB81F980939B
:104600004F029923A9F080914F02816080934F025D
:104610000FC080914F0283FB222720F991E092275F
:1046200090FB83F9ECCF895301C080E00E94742293
:1046300081E0089580E0089580E008950C941C23A3
:10464000CF93C82F80916F02813069F038F08230AB
:10465000C1F58C2F0E94F22181E039C00E94DB104D
:10466000823289F504C00E94DB10823261F48C2F03
:104670000E941E23811104C08C2F0E948B221FC018
:1046800081E090E01CC08C2F0E941C23811116C079
:10469000C43189F058F4CB3089F0C031B1F482E0F4
:1046A00080936F0288E30E94F22108C0C93219F09A
:1046B000C83321F00AC010926F0207C081E08170F8
:1046C00006C010926F0280E002C080E0F8CFCF9168
:1046D0000895CF93DF9386319C4541F5EB010E940D
:1046E000DB10982F8A8120910201309103018823E9
:1046F00079F09A7A81E009F480E080937002911158
:1047000002C069E201C065E3C9010E94FC240AC03D
:1047100080917002811102C069E201C065E3C901A4
:104720000E94FE240E941D1180E001C081E0DF9103
:10473000CF9108950F931F93CF93DF93C42FD22F60
:10474000FC0182818823C9F0409373020E94A32553
:10475000909372028093710280E28C0F883008F08F
:1047600057C0C77081E001C0880FCA95EAF7DF9192
:10477000CF911F910F910C94E5088091730248131B
:1047800030C080917102909172020E94BB25883CDA
:10479000910538F510E21D0FCD17B9F080E28C0FAE
:1047A000883040F4C77081E001C0880FCA95EAF7ED
:1047B0000E94EC08183028F581E09D2F977001C009
:1047C000880F9A95EAF70E94E508802F0E94DC087E
:1047D0001830F0F4D77081E001C0880FDA95EAF75D
:1047E0000AC080E28C0F883098F4C77081E001C065
:1047F000880FCA95EAF7DF91CF911F910F910C9422
:10480000EC08802FDF91CF911F910F910C94DC0861
:10481000DF91CF911F910F9108950F939C01CB01D0
:10482000243F4CE5340731F188F4293DFCE53F078E
:10483000D9F02A3D4CE5340779F1283D3C45A9F5EE
:1048400006E221EE41EE68ED7CE52BC0263FFCE55B
:104850003F07E1F0A8F0273F3C4539F507E225EE98
:1048600046EE67EF7CE51DC007E225EE45EE69EDFB
:104870007CE517C006E221EE40EE64EF7CE511C056
:1048800007E225EE44EE65EF7CE50BC006E221EE83
:1048900042EE66EF7CE505C008E221E045EE6AEDF8
:1048A0007CE50E949A2380E008C0FC018281882375
:1048B00019F01092730201C081E00F910895909356
:1048C000C5018093C4010895909379028093780282
:1048D0000895E0917802F0917902309721F00190EB
:1048E000F081E02D099480E00895E0917802F09144
:1048F0007902309721F00280F381E02D0994089528
:10490000E0917802F0917902309739F022E0DC01F1
:104910002C930480F581E02D09940895209176026E
:10492000309177022817390771F0909377028093BE
:104930007602E0917802F0917902309721F00680BA
:10494000F781E02D09940895209174023091750249
:104950002817390771F09093750280937402E091E3
:104960007802F0917902309721F00084F185E02DF2
:1049700009940895FC01329697E080E0915029F067
:1049800021912223D9F38F5FF9CF0895662349F04F
:10499000FC01329608962191621729F0E817F90771
:1049A000D1F780E0089581E008959C01FC013296E2
:1049B0009FEF80E04191461789F09F3F19F4411124
:1049C00001C0982F8F5F8630A9F79F3F39F0F9011A
:1049D000E90FF11D97FDFA956283089508959C01F2
:1049E0002A5F3F4FFC014281461301C012820196AB
:1049F00082179307B9F708950C94D5240C94EF24EB
:104A0000029626E0FC0111922A95E9F7089508958F
:104A10000C94072583E080937A020C940825811179
:104A200002C081E001C082E080937A020C940825E4
:104A30000C940F2581E080937A020C9408250C9445
:104A40001A2508950C9421250C9422250C942125D7
:104A50000C9421250C942125CF930E9428250E9497
:104A600056160E942625C0E08C2F0E948415892BA3
:104A700029F4CF5FC430C1F780E001C081E0CF915D
:104A8000089508951F920F920FB60F9211248F93DD
:104A90009F93AF93BF9380917B02811113C080914C
:104AA000C4029091C502A091C602B091C70241967E
:104AB000A11DB11D8093C4029093C502A093C602AC
:104AC000B093C702BF91AF919F918F910F900FBE8E
:104AD0000F901F9018958091CC02843031F10E9484
:104AE000330710927B0220E488E190E00FB6F8943F
:104AF000A895809360000FBE2093600083B7817FEC
:104B0000846083BF83B7816083BF7894889583B7BF
:104B10008E7F83BF0FB6F894A8958091600088615E
:104B200080936000109260000FBE08950E94880B71
:104B30000C94370782E084BD93E095BD9AEF97BD52
:104B400080936E0008952FB7F8948091C4029091DD
:104B5000C502A091C602B091C7022FBF08952FB71A
:104B6000F8946091C4027091C5028091C602909140
:104B7000C7022FBF08959C014FB7F8948091C402DB
:104B80009091C502A091C602B091C7024FBF821B8F
:104B9000930B089578941F920F920FB60F921124E1
:104BA0008F939F93AF93BF938091C4029091C5025E
:104BB000A091C602B091C7020196A11DB11D8093BC
:104BC000C4029093C502A093C602B093C702BF91DE
:104BD000AF919F918F910F900FBE0F901F901895DE
:104BE00087E797E790930108809300089AE088E1AF
:104BF0000FB6F894A895809360000FBE9093600064
:104C0000FFCF809187020895089522E02093E90064
:104C10002FEF3091E800215035FD06C035ED3A9573
:104C2000F1F700002111F5CF2091E80025FF0BC01E
:104C300040E050E066E070E00E942F288091E8009C
:104C40008E778093E8000895CF93DF9321E020933F
:104C5000E9002FEF3091E800215035FD06C035ED19
:104C60003A95F1F700002111F5CF2091E80025FFDA
:104C700014C0EC0140E050E068E070E00E942F2892
:104C80008091E8008E778093E80088E0FE01AFE72E
:104C9000B2E001900D928A95E1F7DF91CF910895EE
:104CA00080937C0270937E0260937D028091CC029F
:104CB000843001F582E08093E9008FEF9091E80065
:104CC000815095FD06C095ED9A95F1F70000811190
:104CD000F5CF8091E80085FF0DC040E050E063E033
:104CE00070E08CE792E00E942F288091E8008E7798
:104CF0008093E8000895BC0184E00C945026BC0128
:104D000083E00C9450268091CB02811109C00E944F
:104D1000C0290E941D2A8091E20084608093E200F5
:104D200008951092CB0208950C941F256091C8023B
:104D300081E0611101C080E00C940A259091CC02C1
:104D400081E0943009F080E06091C8020C940F2556
:104D500042E061EC81E00E94392942E261EC82E0AC
:104D60000E9439299091CC0281E0943009F080E0D2
:104D70006091C8020C9418258091CE02833009F40A
:104D800061C030F4813071F0823009F49AC0089526
:104D90008A3009F486C08B3009F46CC0893009F080
:104DA000A8C020C08091CD02813A09F0A2C08091B4
:104DB000E800877F8093E8008091D1029091D20231
:104DC000892B21F468E08FE792E003C060E080E087
:104DD00090E070E00E947A288091E8008B778093C1
:104DE000E80008958091CD02813209F082C080915F
:104DF000D1029091D202029708F07BC08091E80026
:104E0000877F8093E8008091E80082FD05C0809153
:104E1000CC028111F8CF6DC02091F3008091F20097
:104E200090E0922B029731F48091F100813011F0E3
:104E3000863021F48091F100809387028091E80010
:104E40008B7753C08091CD02813A09F052C0809196
:104E5000D1029091D202892B09F04BC08091E800D9
:104E6000877F8093E8008091E80080FFFCCF8091ED
:104E70002B0136C08091CD028132D9F58091D102CB
:104E80009091D202892BA9F58091E800877F8093C9
:104E9000E8000E946E298091CF0280932B010C9430
:104EA000880B8091CD02813221F58091E800877FC7
:104EB0008093E8000E946E298091D002809388023E
:104EC00008958091CD02813AA1F48091E800877F16
:104ED0008093E8008091E80080FFFCCF80918802F9
:104EE0008093F1008091E8008E778093E8000C9425
:104EF0006E29089584B7877F84BF0FB6F894A8956C
:104F000080916000886180936000109260000FBE05
:104F100090E080E80FB6F894809361009093610070
:104F20000FBE0C941A250E94C0290E941D2AE2EE91
:104F3000F0E080818460808378940C94B22C8FE1BF
:104F400091E00C9464248091CC028530A9F4809186
:104F5000CC02853079F40E946B258091CA028823A7
:104F6000B1F30E942C25882391F30E9419280E94F6
:104F7000880BEDCF0C949625089508950C94C027C6
:104F8000292F332723303105C9F060F42130310552
:104F900081F02230310509F044C08BE390E025E137
:104FA0003AE043C021323105E1F02232310549F1C6
:104FB00038C082E190E020E53AE037C0992781309F
:104FC000910549F028F0029761F5E7EDF9E005C099
:104FD000E1E1FAE002C0EFEFF9E0849190E09F0197
:104FE00024C06115710541F061307105D1F489E08B
:104FF00090E020E43AE019C089E090E027E23AE04E
:1050000014C06115710541F06130710551F48BE7F1
:1050100090E022E63AE009C080E490E02DED3AE02D
:1050200004C080E090E020E030E0FA01318320838A
:10503000089580E189BD82E189BD09B400FEFDCFFC
:105040008091D8008F7D8093D8008091E0008260AD
:105050008093E0008091E00081FDFCCF0895CF9225
:10506000DF92EF92FF920F931F93CF93DF93EC01A8
:105070008B017A010E948D29811133C0E114F10462
:1050800039F0F70180819181081B190BC80FD91FD6
:10509000C12CD12C0115110519F18091E80085FD75
:1050A00016C08091E8008E778093E800E114F10447
:1050B00049F0F70180819181C80ED91ED182C0824A
:1050C00085E00FC00E948D29882321F30AC08991B1
:1050D0008093F10001501109FFEFCF1ADF0ADACFF8
:1050E00080E0DF91CF911F910F91FF90EF90DF90C3
:1050F000CF9008952091D3023091D402261737071C
:1051000048F06115710539F42091E8002E7720935D
:10511000E80001C0B901FC0120E06115710579F1D9
:105120008091CC028823F1F18530F1F18091E80083
:1051300083FD3CC08091E80082FD2EC08091E80094
:1051400080FFEBCF2091F3008091F20090E0922B52
:105150006115710551F08830910538F42191209343
:10516000F100615071090196F3CF21E0089709F031
:1051700020E08091E8008E778093E800CECF211167
:10518000CFCF0AC08091CC02882361F0853061F0D6
:105190008091E80083FD0AC08091E80082FFF2CF91
:1051A00080E0089582E0089583E0089581E0089505
:1051B0002091D3023091D4022617370748F06115A9
:1051C000710539F42091E8002E772093E80001C0A2
:1051D000B901FC0120E06115710591F18091CC02CB
:1051E000882309F440C0853009F43FC08091E8006D
:1051F00083FD3DC08091E80082FD2FC08091E800D2
:1052000080FFE9CF2091F3008091F20090E0922B93
:105210006115710559F08830910540F4249120936F
:10522000F1003196615071090196F2CF21E00897A3
:1052300009F020E08091E8008E778093E800CBCFE2
:105240002111CCCF0AC08091CC02882361F0853037
:1052500061F08091E80083FD0AC08091E80082FF40
:10526000F2CF80E0089582E0089583E0089581E020
:105270000895982F973068F59093E900981739F0C2
:105280007091EC002091ED005091F00003C0242FAC
:10529000762F50E021FD02C09F5FECCF3091EB00F4
:1052A0003E7F3093EB003091ED003D7F3093ED0079
:1052B0003091EB0031603093EB007093EC00209361
:1052C000ED005093F0002091EE0027FDE5CF80E047
:1052D00008958F708093E90081E008958091CD0258
:1052E00087FF11C08091E80082FD05C08091CC024B
:1052F0008111F8CF11C08091E8008B770BC08091AD
:10530000CC02882349F08091E80080FFF8CF80919B
:10531000E8008E778093E80008952091E4003091B2
:10532000E50095E64091EC00842F817040FF23C09A
:105330008091E80080FD1DC08091CC02882399F007
:10534000853099F08091EB0085FD11C04091E4001B
:105350005091E5002417350729F3915011F09A0177
:10536000E1CF84E0089582E0089583E0089581E02C
:10537000089580E008954091E80042FFDDCF089550
:105380000E942E2A0E94362AE0EEF0E080818160A1
:105390008083E8EDF0E080818F77808319BCA7EDF2
:1053A000B0E08C918E7F8C9380818F7E8083109271
:1053B000CB0208950F931F93CF93DF930E942E2A61
:1053C0000E94362AC8EDD0E088818F778883888153
:1053D0008068888388818F7D888319BC1092CC0275
:1053E0001092C8021092CA021092C90200EE10E098
:1053F000F80180818B7F808388818160888342E08F
:1054000060E080E00E943929E1EEF0E080818E7F4B
:105410008083E2EEF0E0808181608083808188601B
:105420008083F80180818E7F80838881806188837A
:10543000DF91CF911F910F910895E8EDF0E0808109
:105440008F7E8083E7EDF0E080818160808384E05F
:1054500082BF81E08093CB020C94DA29E8EDF0E082
:1054600080818E7F80831092E20008951092DA008E
:105470001092E10008951F920F920FB60F9211241F
:105480002F933F934F935F936F937F938F939F934C
:10549000AF93BF93EF93FF938091E10082FF0BC026
:1054A0008091E20082FF07C08091E1008B7F8093B2
:1054B000E1000E94B12C8091DA0080FF1FC0809132
:1054C000D80080FF1BC08091DA008E7F8093DA00C5
:1054D0008091D90080FF0DC080E189BD82E189BD46
:1054E00009B400FEFDCF81E08093CC020E948326A8
:1054F00005C019BC1092CC020E9491268091E10057
:1055000080FF19C08091E20080FF15C08091E20009
:105510008E7F8093E2008091E20080618093E200C0
:105520008091D80080628093D80019BC85E0809378
:10553000CC020E9496268091E10084FF30C08091C9
:10554000E20084FF2CC080E189BD82E189BD09B4FD
:1055500000FEFDCF8091D8008F7D8093D800809190
:10556000E1008F7E8093E1008091E2008F7E809346
:10557000E2008091E20081608093E2008091C802A5
:10558000882311F084E007C08091E30087FD02C00A
:1055900081E001C083E08093CC020E949E2680912E
:1055A000E10083FF29C08091E20083FF25C0809144
:1055B000E100877F8093E10082E08093CC0210922B
:1055C000C8028091E1008E7F8093E1008091E2002B
:1055D0008E7F8093E2008091E20080618093E20000
:1055E00042E060E080E00E9439298091F00088600C
:1055F0008093F0000E949426FF91EF91BF91AF91AC
:105600009F918F917F916F915F914F913F912F91DA
:105610000F900FBE0F901F9018951F920F920FB60C
:105620000F9211242F933F934F935F936F937F9328
:105630008F939F93AF93BF93CF93DF93EF93FF939A
:10564000C091E900CF708091EC00D82FD17080FD1F
:10565000D0E81092E9008091F000877F8093F000FD
:1056600078940E94512B1092E9008091F00088609C
:105670008093F000CD2BCF70C093E900FF91EF91A4
:10568000DF91CF91BF91AF919F918F917F916F915A
:105690005F914F913F912F910F900FBE0F901F90F0
:1056A00018951F93CF93DF93CDB7DEB7AA970FB6A8
:1056B000F894DEBF0FBECDBFEDECF2E08091F100BB
:1056C000819322E0E53DF207C9F70E94BC26809154
:1056D000E80083FF2EC18091CD029091CE02492F28
:1056E00050E04A30510508F024C1FA01EE59FF4F4D
:1056F0000C94252D803821F0823809F01AC108C099
:105700008091C9029091CA02992389F082600FC0EA
:105710008091D1028F70873008F00BC18093E9002F
:105720008091EB0085FB882780F91092E900909129
:10573000E800977F9093E8008093F1001092F100C9
:10574000D1C0282F2D7F09F0F4C0882319F08230B2
:1057500061F0EFC08091CF02813009F0EAC0933050
:1057600009F080E08093CA022EC08091CF0281119F
:105770002AC08091D1028F702FEF280F263008F0B9
:10578000D8C08093E9002091EB0020FF1CC093302B
:1057900021F48091EB00806214C09091EB00906145
:1057A0009093EB0021E030E0A90102C0440F551FA7
:1057B0008A95E2F74093EA001092EA008091EB00AC
:1057C00088608093EB001092E9008091E800877F69
:1057D0008093E8000E946E29ACC08111AAC010918C
:1057E000CF021F778091E3008078812B8093E300C4
:1057F0008091E800877F8093E8000E946E29809165
:10580000E80080FFFCCF8091E30080688093E30094
:10581000111102C082E001C083E08093CC0289C0F4
:105820008058823008F085C08091CF029091D002DC
:105830008C3D53E0950779F583E08A838AE289837A
:105840004FB7F894DE01139620E03EE051E2E32FDB
:10585000F0E050935700E49120FF03C0E295EF7011
:105860003F5FEF708E2F90E0EA3010F0C79601C0D6
:10587000C0968D939D932F5F243149F74FBF809140
:10588000E800877F8093E8006AE270E0CE0101962D
:105890000E947A2816C06091D1027091D202AE01A6
:1058A0004F5F5F4F0E94BE27BC01892B09F441C0A6
:1058B0009091E800977F9093E80089819A810E94F7
:1058C000D8288091E8008B778093E80032C0803838
:1058D00081F58091E800877F8093E8008091C8027D
:1058E0008093F1008091E8008E7772CF811121C002
:1058F0008091CF029091D00299270297D4F48091A1
:10590000E800877F8093E8008091CF028093C802EF
:105910000E946E298091C802811106C08091E30027
:1059200087FD02C081E001C084E08093CC020E9428
:10593000A8268091E80083FF0AC08091E800877F55
:105940008093E8008091EB0080628093EB00AA9640
:105950000FB6F894DEBF0FBECDBFDF91CF911F9180
:1059600008950895CF938091CC028823A1F0C0912F
:10597000E900CF709091EC00892F817090FD80E854
:10598000C82B1092E9008091E80083FD0E94512B02
:10599000CF70C093E900CF91089587FB082E0626AB
:1059A00087FD819567FD61950E945C2D0EF49195B0
:1059B00007FC81950895AA1BBB1B51E107C0AA1FD4
:1059C000BB1FA617B70710F0A61BB70B881F991FA0
:1059D0005A95A9F780959095BC01CD01089597FB44
:1059E000072E16F4009407D077FD09D00E94DB2C17
:1059F00007FC05D03EF4909581959F4F08957095D2
:105A000061957F4F0895A1E21A2EAA1BBB1BFD01D1
:105A10000DC0AA1FBB1FEE1FFF1FA217B307E4078D
:105A2000F50720F0A21BB30BE40BF50B661F771FE5
:105A3000881F991F1A9469F76095709580959095C5
:105A40009B01AC01BD01CF010895EE0FFF1F059032
:105A5000F491E02D09940E94332D332312F48A1B14
:105A60009B0B0C94442DA29FB001B39FC001A39F38
:105A7000700D811D1124911DB29F700D811D112487
:105A8000911D08950E94332DB7FF0895821B930B3B
:105A900008950E94332DA59F900DB49F900DA49F53
:105AA000800D911D11240895B7FF0C94492D0E947B
:105AB000492D821B930B0895991B79E004C0991F0F
:105AC000961708F0961B881F7A95C9F78095089558
:105AD000FC014150504030F001900616D1F731974B
:105AE000CF010895882799270895FB01DC0104C0A0
:105AF0008D910190801921F441505040C8F7881BC6
:105B0000990B0895F999FECF92BD81BDF89A992716
:105B100080B50895A6E1B0E044E050E00C94BC2DBF
:105B2000A8E1B0E042E050E00C94BC2D262FF9999A
:105B3000FECF92BD81BDF89A019700B4021639F0EC
:105B40001FBA20BD0FB6F894FA9AF99A0FBE0895BD
:105B50000396272F0E94972D0E94962D252F0E9495
:105B6000972D242F0C94972D0196272F0E94972D67
:105B70000C94962DDC01CB01FC01F999FECF06C0F7
:105B8000F2BDE1BDF89A319600B40D9241505040FB
:085B9000B8F70895F894FFCF67
:105B9800C8003502280850011E0A1401010102003C
:105BA8000C000C0C01191A1B1C1D1E1F20212201A0
:105BB80026242605267F267B26042601E200E90006
:105BC800EA00B500B600B700CD008301CC008A0119
:105BD80092019401210223022402250226022702AF
:105BE8002A02B300B4006F007000818283E200E9EA
:105BF80000EA00B500B600B700CD008301CC008AEA
:105C0800019201940121022302240225022602277F
:105C1800022A02B300B4006F007000818283949757
:105C2800C6343536323331F7F6F5F4939291900055
:105C380001020202020606060909090909090F0FED
:105C48000F0F0F0F151515181919191919191919F1
:045C580019192324CF
:00000001FF
